:10000000E07F0010CD000000F91A0000FB1A00008C
:10001000FD1A0000FF1A0000011B00000000000094
:10002000000000000000000000000000511D000062
:10003000531D000000000000551D0000571D00006A
:10004000591D0000591D0000591D0000591D0000D8
:10005000591D00003D080000591D0000591D0000F9
:10006000591D0000591D0000591D0000591D0000B8
:10007000591D0000591D0000591D0000591D0000A8
:10008000591D0000591D0000591D0000591D000098
:10009000591D0000591D0000591D0000591D000088
:1000A000B9140000591D0000591D0000591D000021
:1000B000591D0000591D0000591D0000591D000068
:1000C000591D0000591D0000591D00000D490E4A20
:1000D0000E4B9A423EBF51F8040B42F8040BF8E76E
:1000E00000200B490B4A91423CBF41F8040BFAE750
:1000F0000948804709488047094880470948004720
:10010000FEE70000783600000000001090000010AC
:1001100090000010D80B0010491E00005D1D00006B
:10012000C31700001519000010B5054C237833B92A
:10013000044B13B10448AFF300800123237010BDBA
:1001400090000010000000002836000008B5064BA3
:100150001BB106480649AFF300800648036813B197
:10016000054B03B1984708BD000000002836000089
:10017000940000100000001000000000064B000476
:10018000302240F4A060C3F80822C3F81002D3F86C
:100190000022D206FBD5704700C00050084B000477
:1001A000202240F40070C3F80822C3F81002D3F8EC
:1001B00000229206FBD5024BD3F81402C0B270475E
:1001C00000C0005010229040054B40F48070C3F8EE
:1001D0000822C3F81002D3F80022D206FBD57047DC
:1001E00000C0005010B5044672B6D020034B9847AB
:1001F00044F08000024B984762B610BD7D010000BC
:10020000C501000010B5044672B6D820034B9847CC
:100210002046034B984762B610BD00BF7D01000029
:10022000C501000010B5044672B6F320034B984791
:100230002046034B984762B610BD00BF7D01000009
:10024000C501000010B5044672B6FE20034B984766
:100250002046034B984762B610BD00BF7D010000E9
:10026000C501000008B572B6FE20034B9847034B4A
:10027000FE20984762B608BD7D0100009D01000088
:1002800010B572B600F00F04C00940EA44042046DD
:10029000034B98472046034B984762B610BD00BFFA
:1002A0007D0100009D01000072B600F00F03C0093F
:1002B00040EA4300012303FA00F0064BC3F838027A
:1002C000D3F800229206FBD5024BD3F8140262B693
:1002D000C0B2704700C0005010B50C4672B600F0B6
:1002E0000F03C00940EA430040F04000034B984729
:1002F0002046034B984762B610BD00BF7D01000049
:10030000C501000008B572B6F220034B9847034BB5
:10031000F220984762B608BD7D0100009D010000F3
:1003200008B572B6FA20024B984762B608BD00BF06
:100330007D01000008B5044B984740F00100C0B2B1
:10034000024B984708BD00BF65020000450200004F
:1003500008B5034B9847034B00F0FE00984708BDD3
:10036000650200004502000037B5324B0446012209
:10037000002002291A708DF804008DF803002E4B1E
:1003800004D1032C3BD118602C480DE029B9012C75
:1003900035D103221A602A4A20E00A2909D10B2C00
:1003A0002DD1022018602748274B8DF802201860B5
:1003B00029E00F2904D1102C21D11A602348F3E73A
:1003C000192905D11A2C1AD103221A601C48EBE70F
:1003D000402909D1412C12D11A601C4A1A4B1A60CB
:1003E00002238DF802300EE0482904D1492C06D1B1
:1003F00002221A60D7E79C2901D19D2CE3E74FF038
:10040000FF321A6014E0C1F34213684601F01F0185
:100410000F4D8DF800308DF80110A847C4F342133A
:10042000684604F01F048DF800308DF80140A8479D
:1004300003B030BDD8040010C802001000C0004056
:1004400000C0094000800940D404001000000140B1
:10045000791F0000904B2DE9F04F00241C708F4B4A
:100460008F4F5A685C601A681C608E4B8BB05A685C
:100470005C601A681C608C4BB8428CBF0127032754
:100480001B684FEA001B08930794A4460294224677
:100490000899CDF80CB021FA07F34FEA43095B0144
:1004A000CDF810900993CDF804900126DDF80C806A
:1004B0000025DDF80490B9FBF8F301335B08B3F5D0
:1004C000803F41D2002B08BF012315B1012B08BF8B
:1004D000022329035943DDF824A0B1FBF6F101EB17
:1004E0000339BAFBF9F94FEAC90181422DBFC0EBCC
:1004F0000109C1EB000ACDF814A0CDF81490824296
:100500002BBFC0EB0209C2EB000ACDF81890CDF862
:1005100018A0DDF81490DDF818A0D14514D2FAB275
:100520001FFA83FC8142F3B202920793ECB22BD004
:100530002CBFC0EB0103C1EB00034FF4C062534377
:10054000B3FBF0F303B30A460135B542D844B0D348
:10055000DDF80C90DDF804A004990136D9448A44F2
:10056000102ECDF80C90CDF804A09FD182422CBF64
:10057000C0EB0203C2EB0003C8214B43B3FBF0F313
:1005800013B1013F032F83D9029A022A96BF474B2A
:1005900003239B5C464A1268032A47D8DFE802F02F
:1005A00002132435434AD2F8C41041F00801C2F8BE
:1005B000C410D2F8A81121F0C00141EA8313C2F897
:1005C000A831052233E03B4AD2F8C41041F01001B3
:1005D000C2F8C410D2F8A81121F4407141EA0323F3
:1005E000C2F8A831062222E0324AD2F8C41041F003
:1005F0008071C2F8C410D2F8AC1121F4403141EA44
:100600000343C2F8AC31072211E02A4AD2F8C410E1
:1006100041F00071C2F8C410D2F8AC1121F44021AD
:1006200041EA8343C2F8AC31082200E0FF22224BAA
:10063000DDF81CA01B6804F00F04197B44EA0A14BF
:1006400041F0800119734FEA1C215FFA8CFC19718B
:1006500083F800C0197BE4B201F07F011973072110
:1006600083F82840197203211973002183F824109C
:1006700093F8301041F0800183F8301051B201231B
:1006800002F01F0203FA02F20C4B490943F8212041
:100690000BB0BDE8F08F00BFC4020010CC02001008
:1006A0003F420F00BC0000108C00001054350000C9
:1006B000C802001000C00F40D404001000E100E0A8
:1006C00010B5034B144698472046024B984710BD7F
:1006D0006903000055040000094B1B68032B0ED86A
:1006E000DFE803F002040608202205E0402203E0D0
:1006F000802201E04FF48072024BC3F880207047E3
:10070000C802001000E100E0064B1B681B7D5B0681
:1007100006D4054B18685B68C01AC0F30800704720
:1007200000207047D4040010CC020010F8B51A4D18
:10073000012128680022194EB0472868184B9847B5
:100740000128FAD0144B1868164B1A6859684A40A9
:10075000C2F308026AB15A685C68511C59601A44B5
:10076000127AD2B202705A685968C2F308025A600B
:10077000EAE71A685C680C4F5440C4F308042CB9CB
:10078000286801212246B0473C70F8BD0121286845
:100790000A463970B047F8BDD40400106921000042
:1007A000C7210000CC020010C402001030B50E4B6F
:1007B00019680B7DDB0716D50C4B08785C681A6846
:1007C000C0B201326240C2F30802002AF1D01A68B6
:1007D0001D68541C1A441C6010721A681868C2F311
:1007E00008021A60E5E730BDD4040010BC00001018
:1007F00038B50D4C0D4B2068984700F00E05062DBE
:1008000006D120680A4B984710F09E0F0AD0FEE7E9
:1008100000F00600042801D1064B9847022D01D1B3
:10082000054B984738BD00BFD4040010BB21000021
:10083000B5210000AD0700002D07000008B5014BF1
:10084000984708BDF1070000014B1860704700BFD2
:1008500030050010054A002353701370044A02212A
:10086000117153719371D371704700BFEE04001082
:10087000DC040010F0B51B4A1B4B94891B68250A49
:100880000021E4B2187828B35E78AE4220D16E1E03
:10089000042E0BD8DFE806F003060A090900002140
:1008A0000C4603E05C79214600E09978A1420ED124
:1008B000022D136008BF5B880A490CBF4B6048607B
:1008C000138A52689A420BDD064A5360F0BD01312B
:1008D0000344D7E70123107150719071D0711372E6
:1008E000F0BD00BFDC0400103005001008B5012089
:1008F000014B984708BD00BF05020000044B0121D1
:100900001970044B002219715A719A71DA7170478B
:10091000EE040010DC04001008B50448837A13F0DC
:100920007C0F01D0024B984708BD00BFDC040010CB
:10093000611C000010B51C4C0020214608221B4BF6
:10094000984708282ED1A4F10A0000234372184BBF
:1009500044F80A3C038A4360837A13F07C0F1FD16A
:10096000C27A092A19D8DFE802F0051D181D1807F8
:10097000111D13150F4B0EE080890F4BC0B2984725
:1009800000210A460D4B8020984710BD0C4B02E019
:100990000C4B00E00C4B984710BD0C4B984710BD1A
:1009A0000B4B984710BD00BFE6040010CD120000AD
:1009B000EE04001055080000E50100004913000096
:1009C00075080000FD080000ED080000BD130000E0
:1009D000FD1B000070B5174C637A53BBA37A6568A2
:1009E000DE091CD095B1412D34BF2A464022124B5E
:1009F000802021689847636822681B1A024463605C
:100A00002260B3B9402814D1267270BD237A83B115
:100A1000802029462A46084B9847257270BD45B963
:100A2000054B802029462A46984701236372034BD1
:100A3000984770BDDC04001049130000190900003C
:100A400010B5164C637A1BBBA07A6268C00911D13D
:100A5000134B52B1216898476368984215DC1B1A02
:100A6000636023681844206010BD10461146984703
:100A700098B10AE04AB910461146094B984720B987
:100A800001236372074B984710BD074B984710BD71
:100A9000002006494022024B984710BDDC0400109C
:100AA000CD12000019090000BD130000EE04001073
:100AB00008B5014B984708BDF11FFF1F38B5044624
:100AC00072B6064833254160C3600549054B056091
:100AD00082600461984762B638BD00BF34050010DB
:100AE00048050010B10A000010B5054B34241C6005
:100AF00058609960DA6018460249034B984710BD68
:100B00003405001048050010B10A000010B5054B6F
:100B100032241C6058609960DA6018460249034B21
:100B2000984710BD3405001048050010B10A0000B8
:100B300070B5054672B604240F2C03D8230303F6C0
:100B4000FF7303E0E303A3F5D023013B994218D2DE
:100B50000F2C85BF04F5FF3303F5F9732303DB0383
:100B600099420A4E08D1204621462A46B0472046DF
:100B700021462A46064B9847204621462A46B0473A
:100B800002E001341E2CD7D162B670BD0D0B0000FF
:100B9000E90A00002DE9F0411B4E336803B93060CB
:100BA0001A4800230468934205D0194DCF5C2544B0
:100BB000EF540133F7E704681C44B4F5007F046088
:100BC0001ED1DFF85C803168D8F800004FF47A77E6
:100BD000104EB0FBF7F0104B984730680A4D80B9C3
:100BE000D8F800002346B0FBF7F02968084A0B4C00
:100BF000A047306828B9054B28601860BDE8F0812F
:100C00000020BDE8F08100BFAC000010B000001073
:100C10005C05001048050010310B0000BD0A000003
:100C20008C0000100131002370B5891A0546184662
:100C30008B420DDA9C18A5EBE406F67B04F0070462
:100C400046FA04F404F001049C4001332043EFE72A
:100C500070BD000010B51C46064B98472046064B59
:100C600098472046054B9847054B20469847054B2B
:100C70001C8010BD41150000051700002D17000055
:100C80004D17000064070010034B1868D0F10100F5
:100C900038BF0020704700BF6C070010014B186878
:100CA000704700BF6C0700104FF4007070470000E1
:100CB0002DE9F0411A4F1B4B0446B7F900000D46D1
:100CC000984744F04000C0B2174CA047280EA047F8
:100CD000C5F30740A047C5F30720A047E8B2A047E7
:100CE0009520A0474FF48055FF20A04710F0800FBB
:100CF0000D4E804608D1B7F900000C4B9847FF20F5
:100D0000B0474046BDE8F081013DEDD1B7F90000A4
:100D1000064B9847FF20B0474FF0FF30BDE8F08109
:100D20006407001065170000B11600004D170000A1
:100D300038B54FF4805400213720074DA8472920AB
:100D40000021A84718B9054B0120186038BD013CA7
:100D5000F1D1204638BD00BFB10C0000680700107B
:100D600070B5154E154B0446B6F900000D46984770
:100D700044F04000C0B2124CA047280EA047C5F373
:100D80000740A047C5F30720A047E8B2A047952039
:100D9000A0474FF48055FF20A04703060AD5013D28
:100DA000F9D1B6F90000074B9847FF20044B98474C
:100DB0004FF0FF3070BD00BF6407001065170000E2
:100DC000B11600004D1700002DE9F843214D224BCC
:100DD0000646B5F900009847204C7A20A04700202D
:100DE000A0470020A0470020A0470020A047952052
:100DF000A0474FF48057A846FF20A04710F0800F6F
:100E0000164D81461AD1FF20A84704063460FF2002
:100E1000A84744EA00443460FF20A84744EA00247D
:100E20003460FF20A847204330600D4BB8F9000024
:100E30009847FF20A8474846BDE8F883013FDBD12B
:100E4000B8F90000064B9847FF20A8474FF0FF3045
:100E5000BDE8F8836407001065170000B1160000B4
:100E60004D17000037B54FF48054002137200D4D49
:100E7000A84729204FF08041A84758B90A4B01A83C
:100E80009847019B13F0804F084B14BF03200220AA
:100E9000186004E0013CE8D1044B20461C6003B01C
:100EA00030BD00BFB10C0000C90D00006807001084
:100EB00073B51C4E1C4BB6F9000098471B4C4820DC
:100EC000A0470020A0470020A0470120A047AA205B
:100ED000A0478720A0474FF47A15FF20A0470306BC
:100EE0008DF8000011D40125FF20A0470DF8050062
:100EF0000135052DF8D1B6F900000D4B9847FF20BC
:100F00000A4B98479DF800000AE0013DE5D1B6F98B
:100F10000000074B9847FF20044B98474FF0FF30E5
:100F200002B070BD6407001065170000B116000024
:100F30004D17000010B546F2A810114B9847114B01
:100F40001024B3F90000104B9847FF200F4B98472F
:100F5000013CFAD1204621460D4B984701280AD181
:100F60000C4B9847012801D10B4B02E0052802D118
:100F70000A4B984710BD0A4B20461C6010BD00BFAD
:100F8000CD140000640700104D170000B1160000DA
:100F9000B10C0000B10E0000650E0000310D000024
:100FA000680700102DE9F041114C8046114BB4F94F
:100FB00000000F4698472646FF200F4CA047FE280A
:100FC000FAD10025BD424FF0FF0004DAA04708F82F
:100FD00005000135F6E7A047FF20A047B6F900005D
:100FE000064B9847FF20A0470020BDE8F08100BFD6
:100FF0006407001065170000B11600004D170000CF
:1010000038B50C4B05461B685A1E012A01D8490207
:1010100002E0032B18BF00211120074B984704461C
:1010200028B928464FF40071044B984700E001248A
:10103000204638BD68070010B10C0000A50F000065
:101040002DE9F041194E1A4B8046B6F900000F46C3
:10105000184C9847FE20A0470025BD4204DA18F836
:101060000500A0470135F8E7FF20A047FF20A04773
:10107000FF20A04700F01F00052809D0B6F90000A6
:101080000D4B98470B4BFF2098470120BDE8F0819E
:10109000FF20A0470028FBD0B6F90000064B984778
:1010A000044BFF2098470020BDE8F0816407001042
:1010B00065170000B11600004D17000038B50C4B45
:1010C00005461B685A1E012A01D8490202E0032B7B
:1010D00018BF00211820074B9847044628B9284616
:1010E0004FF40071044B984700E00124204638BDBE
:1010F00068070010B10C0000411000007FB5092006
:101100000021204B984708B1002038E068461021A4
:101110001D4B98470028F7D168467F217E221B4C43
:10112000A04700BB1A4B1B68032BEDD049213E2280
:101130006846A047312105462F226846A047502225
:10114000064653216846A0470236012202FA00F300
:10115000B24005FB0220B3F5007F33BF58435B0A62
:101160005843400A0BE00128CED1094B1B68032BE2
:10117000CAD1684645213022A0470130800204B020
:1011800070BD00BF610D0000A50F0000250C000020
:101190006807001010B50C4C002323600B4B9847D8
:1011A00008B901240DE00A4B98474FF40071206004
:1011B000084B1020984704460028F2D10648074BF8
:1011C0009847204610BD00BF6C070010350F000087
:1011D000FD100000B10C000000093D00CD1400001E
:1011E00010B5134BD3F8C42042F00042C3F8C4201A
:1011F000104BD3F8F42F42F01202C3F8F42FD3F8B7
:10120000F82F122AFBD10C4C636823F070536360F3
:10121000636843F0A0536360084B9847236923F445
:1012200040332361236943F48023236110BD00BF51
:1012300000C00F4000C0005000C002405103000039
:1012400008B5014B984708BD5103000010B572B6B0
:10125000124B4FF48072C3F8082200F00F02C0094D
:1012600040EA420001228240D3F844421443C3F8CA
:101270004442C3F84802C3F84C1262B60748D0F89B
:101280000012064BC905FAD54FF48071C3F8081255
:10129000D3F834120A43C3F8342210BD00C0005002
:1012A00010B5074B0C22C3F80422064C80204021C5
:1012B000A04700204021A047034B984710BD00BF26
:1012C00000C000504D1200003503000070B572B62A
:1012D00000F00F04194BA40044F00104C3F82842A5
:1012E0001D46D5F82042154B2405FAD5D3F82052D7
:1012F000C5F3090595421EDC15B1002423460EE016
:10130000D3F8183213E013F0030604BF0B4CD4F8E3
:101310001842032ECC544FEA142403D001339342D5
:10132000F1DB04E0054ED6F82862F607F6D4044B4C
:101330009847044B984762B6284670BD00C00050DD
:101340008102000005030000F8B5154672B600F0F2
:101350000F02174B920042F00202C3F82822C3F892
:101360002452B5B10024124AD2F828329B0713D573
:10137000AC4211DA0B199E785F78360446EA0726EC
:101380000F5DDB783E4346EA0363C2F81C32043447
:10139000E9E7C3F81C522C46064B9847064B984782
:1013A000BFF36F8F62B6AC42B4BF20462846F8BD8B
:1013B00000C00050810200002103000008B5002099
:1013C0008021014B984708BDD902000037B5304B4A
:1013D000D3F80022D20744BF0122C3F80822D3F871
:1013E00000321B0713D52A4B0822C3F80822294BC9
:1013F0009847C5060BD5284B9847284C802040219C
:10140000A04700204021A0470220254B9847204BB1
:10141000D3F80022540738D5D3F83042E00710D56E
:101420000020204B9847410701D51F4B03E010F0E7
:10143000010002D01D4B984703E0694608221C4B6F
:101440009847A20706D5174B80209847C30701D4B9
:10145000184B984734F0030304D10D4B0422C3F812
:10146000082212E008250324094BD3F830321D422C
:1014700005D0E00140EA6400C0B20A4B984701344D
:10148000202C4FEA4505EFD1E7E703B030BD00BFA0
:1014900000C0005065020000151D00004D12000044
:1014A00025020000A902000035090000410A0000E1
:1014B000CD120000D5090000684620F007018D46D6
:1014C00001B5BDE80140854670470000184A194B38
:1014D000B2FBF0F21A60184B1B6843B3B0F5C07F43
:1014E0000AD81A69FE221A611A681968D2B21A60FB
:1014F0001A6842F47F4218E01049884205D91A69F7
:1015000002221A611A68D2B20FE002F0FE011869D5
:10151000196119681868C9B2196019681869B2FBAD
:10152000F0F2013A120292B20A4319681A60704747
:1015300040787D01780700107007001020BCBE00C5
:101540002DE9F04101270D4600F01F011446DFF898
:101550005C81064607FA01F1C0F342103A46C047E3
:1015600005F01F01C5F3421007FA01F10022C04740
:1015700004F01F013A46C4F3421007FA01F1C047D4
:10158000092E444A22D1082D60D1072C5ED1424B4E
:101590001360A3F58043196821F47C211960196850
:1015A00041F42821196003F55023D3F8A81121F440
:1015B0004011C3F8A811D3F8A81141F48011C3F861
:1015C000A811D3F8C41041F480612BE0122E2CD165
:1015D000112D3BD10F2C39D1304B1360A3F5B8231B
:1015E000196821F040411960196841F00041196003
:1015F000596821F03C015960596841F0280159604F
:1016000003F55023D3F8AC1121F44061C3F8AC11B9
:10161000D3F8AC1141F48061C3F8AC11D3F8C41015
:1016200041F40011C3F8C41012E0382E0ED1372D4A
:101630000CD1342C0AD1194B19491360CB6843F4EF
:10164000703343F44073CB60164BDBE70023136029
:101650001368E3B11A681968120C12041A601A6848
:10166000196842F007021A605A68596822F00F029E
:101670005A605A6842F2107059685A600A4B98478B
:10168000044B1B685A68596842F002025A60BDE870
:10169000F08100BF70070010000003400080084088
:1016A00000C0024000C00F40CD1400008D2000009B
:1016B000074B1B6853B1DA689107FCD59A689860AC
:1016C000DA685207FCD59868C0B270471846704770
:1016D0007007001007B500238DF802308DF8043034
:1016E0008DF80330C0F3421300F01F008DF8003076
:1016F0008DF80100024B6846984703B05DF804FB83
:10170000791F000008B5014B984708BDD5160000A9
:1017100008B50A4600F01F0301219940C0F34210AA
:10172000014B984708BD00BF8D20000008B501217E
:10173000014B984708BD00BF1117000008B50021F4
:10174000014B984708BD00BF1117000008B50121E3
:1017500000F01F039940C0F34210014B984708BDA9
:101760009920000008B5012100F01F039940C0F343
:101770004210014B984708BDA520000038B504462B
:101780000D46044B984720460DB1034B00E0034B38
:10179000984738BD2D1700004D1700006517000051
:1017A00010B5064B0446C0F34210984704F01F04DE
:1017B000E04040F30000C0B210BD00BFB120000007
:1017C000704770470020704782B000230093009B51
:1017D000834204D2009B0193009B0133F6E70198FA
:1017E00002B0704738B5C5B20A4C05F0010132208D
:1017F000A04705F002013320A04705F00401342082
:10180000A04705F008013520A0479C2005F01001F5
:10181000A04738BD7D17000008B54C20014B984704
:1018200008BD00BFA117000008B5074B9847074B3C
:101830009847074B9847074B984708B9064BF9E775
:10184000064B984708BD00BF051B0000E1110000D2
:10185000A1120000011D0000CD1300004112000084
:10186000F0B5204CADF5037D1F49204B0020984773
:101870001F48216801221F4B9847264600282ED179
:101880004FF4007301934FF48044019D1848B5F55F
:10189000007F16D102A92A4601AB174FB84718B1ED
:1018A000164B134898471AE0A4F58040C00B144B20
:1018B00098472046134B02A92A469847019B1C448F
:1018C000E3E70E4B9847B4F5804F08D90E4D0F4B08
:1018D00028689847296801900D4B306898470DF5A6
:1018E000037DF0BD040000107E070010B92E00003B
:1018F000AC090010D92E0000413000002D3200004C
:10190000E5170000950B00000800001045320000AC
:101910001D33000073B5614B614C98474C20A047C4
:10192000604B4C20984732205F4DA0473220A8479B
:101930003320A0473320A8473420A0473420A847AD
:101940003520A0473520A8479C20A0479C20A847C9
:101950004420A0474420A847544E00214420B047CB
:101960004520A0474520A84700214520B0474620F4
:10197000A0474620A84700214620B0474720A0475F
:101980004720A84700214720B0471F20484B9847D1
:10199000484B03200221484A98474FF48053019353
:1019A000019B13B1019B013BF9E7062309200821A4
:1019B0000722424CA047424B984708B9414B9847F1
:1019C000414B9847002866D0404B984710B1404B98
:1019D000984760E04FF480431B6801335BD03D4C77
:1019E000A0470028FBD1A0470028FCD13A4B9847DC
:1019F0003A4C3B48A0473B4B4FF480429A603A4BED
:101A00000122C3F88020AA22C3F88C205522C3F8F3
:101A10008C20D3F88810344A11F00071F9D1AA2330
:101A2000C2F88010C2F88C305523C2F88C302E4A90
:101A3000D2F8883013F08073F9D1C2F8A030AA230D
:101A4000C2F8AC305523C2F8AC30D2F8A810264BFF
:101A500011F40071F9D11A684FF47A70C2F30B02D5
:101A60001A601A6842F4A0421A60C3F80411C3F85D
:101A70000C11C3F8A011A047BFF35F8FBFF34F8FC6
:101A8000BFF36F8F4FF480431B6883F3088844F2E1
:101A900004031B689847154B9847A0E7572100009F
:101AA000051700003D1700002D1700007D170000EE
:101AB000E5170000C106000040420F00550C000071
:101AC0009511000061180000191800003D21000068
:101AD0004921000009070000D9060000C9170000CD
:101AE000C0C62D0000ED00E000C00F402918000026
:101AF00000487047A1A16DB9FEE7FEE7FEE7FEE7EB
:101B0000FEE7000008B50348034B9847034A044B1F
:101B10001A6008BD0C0000104908000000400000D9
:101B2000D40900100D4B81890360038A0C4A43607D
:101B30000C4802EB412101607BB10B440A490A4485
:101B400093420A490A4B03D803220A70052203E094
:101B50000A220A70082119701A717047D8090010FA
:101B600000400000D409001000C00700D009001098
:101B7000850000100D4B092230B51A7083890C497D
:101B80000C4A01EB43231360028A0B4D9C18294435
:101B90008C4202D80360426030BD00230371437160
:101BA0008371C3710123037230BD00BFD0090010DF
:101BB00000400000D409001000C00700044B0022C0
:101BC0001A7002221A71034A034B1A60704700BF51
:101BD0008500001000400000D4090010044B0022D2
:101BE0001A7002221A71034A034B1A60704700BF31
:101BF0008500001000400000D409001008B5837A69
:101C000003F07F03212B1ED1C37A013B052B1AD889
:101C1000DFE803F00305070C0E170B4B12E00B4B2C
:101C200010E00B4B06220360002305E0094B09E09E
:101C3000094B012203600023027143718371C37158
:101C400008BD064B984708BD251B0000751B00000A
:101C500085000010BD1B0000D0090010DD1B000036
:101C600070B5837A044603F07F03212B39D1C37A00
:101C7000022B2ED0032B02D0012B32D108E0194BBE
:101C8000194A1B79082B13702BD1184B984770BD3C
:101C9000038A144DBBB1164E164B3068A0F5804038
:101CA000C00B9847306814494FF40072134B9847A3
:101CB00028B9228A336813443360052307E00623DA
:101CC0002B700A2303E0084B06221A7008232B719D
:101CD00070BD044B09221A71054B018A1A680A4427
:101CE0001A6070BD85000010D0090010411200007C
:101CF000D4090010E5170000D8090010950B00006A
:101D0000034B1878B0F1080358425841704700BFA0
:101D1000D009001008B50A4B1B78063B022B0DD8E2
:101D2000084B9847BFF34F8F074A084BD16801F41F
:101D3000E0610B43D360BFF34F8FFEE708BD00BFE8
:101D4000D00900104112000000ED00E00400FA0587
:101D5000FEE7FEE7FEE7FEE7FEE7000008B5064BFC
:101D60009847064B98470648064B984708BDFEE73C
:101D7000FEE7FEE7FEE7FEE7BD200000F1200000E1
:101D8000000000003121000010B5294BD3F8882055
:101D9000D3F80C11C2F30162032A01F00301254AB2
:101DA00032D101290BD002291AD0D3F88840D3F8B8
:101DB0008800C4F30E04D3F804111F4B08E0D3F8D5
:101DC0008840D3F88800D3F804111C4BC4F30E04E8
:101DD00004FB0333C0F307400130B3FBF0F30EE024
:101DE000D3F88800D3F88840C0F30E00D3F804116C
:101DF0000130C4F3074300040133B0FBF3F3C9B26D
:101E00000131B3FBF1F310E0D3F804310129DBB267
:101E100003F1010303D0022903D0094903E0094972
:101E200001E04FF40041B1FBF3F3136010BD00BFBC
:101E300000C00F408C00001000127A0000366E01C6
:101E400000093D00001BB70010B5444B2022C3F829
:101E5000A021D3F8A02186B0940603D5D3F8A02101
:101E60005006FBD50022C3F8A821C3F8AC210122FB
:101E7000C3F80C210222C3F8042106A8362340F837
:101E8000183D01A9364B68469847029B334C13F422
:101E9000801F08BF334A4FF0AA0318BF0E22C4F8B0
:101EA0008420C4F88C305523C4F88C302B4B01228D
:101EB000C3F88020AA22C3F88C205522C3F88C20B6
:101EC000D3F88810254A4901FAD50323C2F8803097
:101ED000AA23C2F88C305523C2F88C301F4BD3F89C
:101EE000882012F0407FF9D02322C3F8A420AA2131
:101EF00055220120C3F8AC10C3F8AC20C3F8A000F1
:101F0000C3F8AC10C3F8AC20144BD3F8A82052058A
:101F1000FAD50322C3F8A020AA22C3F8AC20552288
:101F2000C3F8AC20D3F8A8200C4C12F4407FF9D0B1
:101F30000D4B98470D4B0E4AC4F8C4300023C4F82B
:101F4000C83145F23A0323600A4B1B6823F0404333
:101F500023F07F03936006B010BD00BF00C00F40A8
:101F6000F11FFF1F18000100891D00000884208058
:101F700000ED00E00000000070B5427884780F2A80
:101F800088BF103A4FEA42024FF0030505FA02F506
:101F900004FA02F203784FF003064FEA430388BFC6
:101FA00001339B0003F1804303F53033196821EAC4
:101FB00005010A431A604278C5780F2A88BF103A93
:101FC0004FEA420206FA02F605FA02F203781249D3
:101FD0004FEA430388BF013351F8234024EA060443
:101FE000224341F823200278417800790B4B0128E5
:101FF00007D100FA01F153F822400C4343F8224084
:1020000070BD012000FA01F153F8220020EA01001E
:1020100043F8220070BD00BF40C0024068C00240CB
:1020200004280CD8064B53F8203043B112B11A687B
:10203000114302E01A6822EA01011A681960704728
:1020400074350000042805D8034B53F820300BB139
:102050009A699961704700BF74350000042805D85B
:10206000034B53F820300BB1DA69D961704700BFD8
:1020700074350000042805D8034B53F8200010B134
:1020800040697047002070477435000008B5014B67
:10209000984708BD2120000008B5014B984708BDAE
:1020A0004520000008B5014B984708BD5D200000A1
:1020B00008B5014B984708BD752000000B4B4FF049
:1020C000FF310122C3F88010C3F88420C3F88011C7
:1020D000C3F88421002303F16042013302F5614219
:1020E0000021202B82F80013F5D1704700E100E0B9
:1020F0000D4B4FF020620D495A6000229A60D96062
:102100001A615A6102F16041013201F56D4100200E
:10211000202A054B0876F5D14FF0FF3258629A62BB
:10212000DA621A63704700BF00ED00E00000FA05B4
:10213000014B9860704700BF00ED00E04FF0804316
:102140001878C0F3800070474FF080431A7802F08F
:10215000FB021A70704772B64FF08043AA221A72BF
:1021600055221A7262B67047062996BF0F4B00239C
:1021700033F81130012A0E4A05D19042426843EAF1
:1021800002030FD10FE090426FEA030305D14268CA
:1021900040F28F3111400B4005E0416840F20732B8
:1021A0000A40134042684360704700BF8835000012
:1021B00000000140007DC0B27047806820F0300010
:1021C0008005800D7047007D80F04000C0F38010D6
:1021D000704710B50023934203D0CC5CC454013344
:1021E000F9E710BD2DE9F843D0F82A5004468D4296
:1021F0000E4602D10020BDE8F883037913B9002E02
:10220000F8D022E000F12E08164F407841462A46C9
:102210000123B847B94610B10120BDE8F883D4F8CE
:102220001A20D4F81E30207113449D42E7D2E7787B
:10223000012FE4D9D4F81A3060781D4441462A466B
:102240000123013FC847FFB2F2E7607804F12E0195
:1022500032460123044DA8470028DDD1C4F82A6086
:10226000BDE8F8839D3400007134000008B50368B0
:1022700073B11A7862B1D9888288914208D15878AE
:10228000044B984710F0010F0CBF0020032008BD3D
:10229000092008BD59340000CA7E8B7E032843EA1A
:1022A000022305D1487D0A7D42EA002243EA024327
:1022B0001846704738B504460A46407804F12E01A6
:1022C00001231C4DA84780BB94F82C3294F82D2292
:1022D00043EA0222184B12B29A4228D194F866209F
:1022E00094F86730120442EA036294F864301A43A7
:1022F00094F8653042EA0322104B22F07F429A4262
:1023000016D094F8820094F88320000440EA02601A
:1023100094F88020104394F8812040EA022020F0B5
:102320007F40C01A18BF012038BD032038BD0220ED
:1023300038BD00BF7134000055AAFFFF464154006C
:102340002DE9F041154602681378303B092B05D87A
:1023500054783A2C02D10232026000E000230022BD
:102360000A60002B40F06A81BD4B1C68002C00F015
:1023700068810C60237873B16078BA4B9847C607C0
:1023800009D4002D00F0608110F0040F0CBF002074
:102390000A20BDE8F081002020706070B24B9847A1
:1023A000C10700F1548115B1420700F15381204665
:1023B0000021AE4DA847012817D194F8F03113B988
:1023C0000D20BDE8F08194F8F66194F8F7313604F9
:1023D00046EA036694F8F43120461E4394F8F5313A
:1023E00046EA03263146A84700E00026032800F00D
:1023F00034810028E4D194F83A2094F8393043EA43
:102400000223B3F5007FDBD194F8450094F8443003
:1024100053EA00200DD194F8540094F8553000048C
:1024200040EA036094F85230184394F8533040EA7D
:10243000032094F83E50C4F81A006B1E012BE5707F
:10244000BED894F83B10A1700029B9D04B1E0B42A6
:10245000B6D194F83F3094F8402043EA02221307A3
:102460002281ADD194F8427094F8413053EA0723A9
:102470000DD194F8503094F851701B0443EA07636F
:1024800094F84E703B4394F84F7043EA072394F856
:102490003D8094F83C7057EA082891D005FB00FC79
:1024A00008EB12176744BB428AD3DB1BB3FBF1F383
:1024B000002B85D040F6F5718B4206D94FF6F575A5
:1024C000AB428CBF0325022500E0012502333744CF
:1024D00006EB0801032DC4F81630C4F82670C4F8C2
:1024E0001E1014D1002A7FF46BAF94F85C2094F88E
:1024F0005D10120442EA016294F85A109B000A43EC
:1025000094F85B1042EA0122C4F8222011E0002A6C
:102510003FF456AF022D4FEA430218BFD218614470
:1025200018BF03F00103C4F822100CBF134603EBDD
:10253000520303F2FF13B0EB532FFFF441AF4FF000
:10254000FF33A373E37323746374032D4FF000030D
:10255000A372E372237363735DD1637194F85F2098
:1025600094F85E30607843EA02223244C4F81220C4
:1025700004F12E0101233E4EB04700284BD194F8C0
:102580002C3294F82D2243EA02223A4B12B29A429C
:1025900041D194F8302094F83130120442EA0362B9
:1025A00094F82E301A4394F82F3042EA0322324B2B
:1025B0009A4230D194F8142294F81532120442EA67
:1025C000036294F812321A4394F8133242EA032257
:1025D0002A4B9A421FD194F81C3294F81D221B04F6
:1025E00043EA026394F81A22134394F81B2243EA45
:1025F0000223C4F80A3094F8183294F819221B0404
:1026000043EA026394F81622134394F8172243EA2C
:102610000223C4F80E301A4A0020138825700133B3
:102620009BB220711380E38084F82A0084F82B0089
:1026300084F82C0084F82D00BDE8F0810B20BDE863
:10264000F0810C20BDE8F0812846BDE8F081032030
:10265000BDE8F0810A20BDE8F0810120BDE8F081ED
:10266000B80000105934000041340000B5220000C9
:102670007134000055AAFFFF5252614172724161EC
:10268000B400001070B5314B002104469847034652
:10269000002B5AD12278032A4FD16279002A4CD0DC
:1026A00084F82A3084F82B3084F82C3084F82D30CC
:1026B00004F12E010025CD540133B3F5007FF9D18B
:1026C000552384F82C32AA2384F82D32522384F81F
:1026D0002E3084F82F30612384F8303084F815329E
:1026E000D4F80E30412284F8312084F81422C3F348
:1026F000072284F8163284F817221A0C1B0E84F86D
:102700001932D4F80A3084F81822C3F30722722051
:1027100084F81A3284F81B221A0C1B0E84F8120259
:1027200084F8130284F81C2284F81D326078D4F8EF
:1027300012200123064EB0476571002160780A46D9
:10274000044B9847003018BF012070BDE521000000
:102750009D340000C9340000D0F816300239023B25
:1027600099423DBF8278D0F8263002FB013000202C
:102770007047000001292DE9F04104460D4666D955
:10278000D0F81630994262D20378022B29D0032B5D
:102790003BD0012B57D101EB5106D0F81E102D4F25
:1027A00001EB5621B84700284DD1D4F81E10C6F3CE
:1027B000080301362344204601EB562193F82E806E
:1027C000B84700283FD1C6F30806344494F82E00D9
:1027D000EB0748EA00204CBF0009C0F30B00BDE83E
:1027E000F081D0F81E101B4B01EB1521984750BB10
:1027F0006D0005F4FF7563192C4493F82E3094F89E
:102800002F0043EA0020BDE8F081D0F81E10114BE4
:1028100001EBD5119847B0B9AD0005F4FE75631909
:1028200093F8310093F830202E335B78000640EAAD
:1028300002402C4440EA032094F82E30184320F044
:102840007040BDE8F0814FF0FF30BDE8F08101201D
:10285000BDE8F081E521000070B50D46C1808168BA
:102860000446012901D1022070BD0368D3F8162067
:102870009142F8D299B91A78032A02D1D3F82210DA
:1028800069B9002222736273A273E2731A89AA42A1
:10289000E9D9D3F8223003EB1513236119E09E78B0
:1028A0003601B54220680ED30F4B9847431C0146B2
:1028B00018D00128D7D92368D3F816309842D2D23D
:1028C000AD1BADB2EDE7E160084B984700EB15108A
:1028D0002061236805F00F0503EB45152E35656172
:1028E000002070BD012070BD752700005927000031
:1028F00010B5084BC1880446984750B92068216933
:10290000054B984728B96369E5221A7023680122AC
:102910001A7110BD59280000E521000001292DE998
:10292000F04104460D46164676D9D0F81630994245
:1029300072D20378022B3AD0032B4AD0012B66D1F6
:1029400001EB5107D0F81E10DFF8D48001EB5721BE
:10295000C04700285CD1C7F3080315F001052344E4
:10296000F2B206D093F82E1001F00F0141EA0212E4
:10297000D2B283F82E20D4F81E1001370123237120
:10298000204601EB5721C047002841D1C7F3080773
:10299000274415B1C6F3071606E097F82E30C6F3A4
:1029A000032623F00F031E4387F82E6030E0D0F893
:1029B0001E101B4B01EB1521984748BB6D0005F419
:1029C000FF75631983F82E60C6F3072683F82F601E
:1029D0001EE0D0F81E10124B01EBD5119847B8B984
:1029E000AD0005F4FE75631993F83120120602F06C
:1029F00070421643C6F3072283F82E6083F82F2017
:102A0000320C360E83F8302083F8316000E002206B
:102A100001232371BDE8F0810220BDE8F08100BFF1
:102A2000E5210000F8B505460F4641B9D0F80A6027
:102A30007EB1D0F816309E4228BF01260AE0234B13
:102A4000984701283FD9D5F8163098423CD33E46E6
:102A500000E001263446D5F8163001349C4204D3F8
:102A6000012E01D80020F8BD022428462146174B2C
:102A7000984748B1411C02D14FF0FF30F8BD012802
:102A800021D0B442E7D1EDE7284621466FF07042ED
:102A90000F4EB047A8B95FB9D5F80E30C5F80A4057
:102AA0005A1C0CD0013BC5F80E3001236B7106E0B7
:102AB000284639462246B0470028EDD001E020469E
:102AC000F8BD0128D8D00120F8BD00BF752700004F
:102AD0001D2900002DE9F047C68804460136B6B22C
:102AE0000F4616B90420BDE8F0870369002BF9D022
:102AF00016F00F0861D1C16801330361006819B98C
:102B00000389B342EED958E08278013A12EA1612EC
:102B100053D1314B98470128054602D80220BDE821
:102B2000F087421C02D10120BDE8F0872068D0F870
:102B300016309D423BD3002FD4D0E168274B9847F5
:102B40000546002844D00128E8D0431CEBD0244F90
:102B500020680021B847B9460028E4D123682E3305
:102B600000271F540130B0F5007FF9D1D4F800A040
:102B7000294650461B4B9847CAF82A002368FAB2E8
:102B8000997891420ED901221A7120680021C84714
:102B900001370028C7D12368D3F82A200132C3F8AF
:102BA0002A20EBE7D3F82A108A1AC3F82A20E56016
:102BB000206829460B4B984720612368E68003EB89
:102BC000481808F12E08C4F814800020BDE8F087EA
:102BD0000720BDE8F08700BF75270000252A000008
:102BE000E5210000592700002DE9F0410B7804464B
:102BF0002F2B0E4601D05C2B00D10136002525720B
:102C00006572A572E57233781F2B4ED8204629468F
:102C10005A4B984725756575A575E575BDE8F08132
:102C20005C2B42D0A56900232022EA5401330B2BF0
:102C3000FAD100208446082102460CF1010C07EB72
:102C40000C0616F8013C202B36D8202B8CBF002315
:102C50000423002874D02878E52804BF05202870B4
:102C6000082904BF9200D2B202F00301012902F048
:102C70000C0208BF43F01003042A08BF43F0080306
:102C8000EB72204600213D4B984760B3A369DB7A85
:102C900000284AD15A076FD46169CB7ADB064CD53C
:102CA00023681878364B9847A060337837462F2B27
:102CB00006F10106B4D1F8E72F2BC6D05C2BC4D0A7
:102CC0002E2B52D088423BD21E0604D52D4E803B7F
:102CD000F35C42F00302DFF8B88018F8016F96B396
:102CE0009E42FAD12CE020682169274B98470028A2
:102CF000CCD162691378B3B1D17A01F0080101F047
:102D0000FF0359B9A569D15C0133E81810F8010C2B
:102D1000884203D10B2BF6D10020B7E720460021D3
:102D20001A4B9847B1E70420B0E7042824D113F0E8
:102D3000040F08BF0520BDE8F0810520BDE8F08143
:102D40000620BDE8F081A3F14106192E02D842F019
:102D5000020207E0A3F16106192E03D8203B42F0DE
:102D60000102DBB22B54013067E70829E8D1920059
:102D70000846D2B20B2160E7BDE8F0815928000077
:102D800099220000A5350000E5210000D52A0000A9
:102D90009535000070B50021144B04469847054650
:102DA00010BB20682169124EB0470546E0B963693F
:102DB0001B78E52B05D023B1204601210D4B984708
:102DC000EDE720682169B047054668B960692B4680
:102DD0000022C2540133202BFAD10B22064BA169E9
:102DE0009847236801221A71284670BD59280000AF
:102DF000E5210000D52A0000D321000010B50423EE
:102E000004462169A1B12068104B9847D0B9626986
:102E10001378B3B1E52B04D02E2B02D0D37A1B0745
:102E200012D5204600210A4B984758B90346E8E7D7
:102E300018464BB1002222746274A274E2741846E0
:102E400010BD04200346F5E710BD00BFE5210000DA
:102E5000D52A0000012970B504460D4626D9D0F8C0
:102E60001630994222D2D4F816309D4205D220461F
:102E700029460F4B9847064608B9002070BD012827
:102E800014D0411C10D0204629460022094B9847F7
:102E900068B9D4F80E305A1C04D00133C4F80E308F
:102EA000012363713546DEE7012070BD022070BD4D
:102EB000752700001D29000048B9064A136803B1B0
:102EC000187009B100230B701160002070470B20AF
:102ED000704700BFB80000102DE9F0438DB001919C
:102EE00016460546002800F09280002303704370C8
:102EF0008370C37005A901A802F01E02494B9847D0
:102F0000002840F08B8002AB0B9305A80199464B3B
:102F100098470A9C10B9002C08BF062016F01C0F19
:102F200006F01F0743D048B1042802D105A83F4B43
:102F3000984747F008070A9C30B16FE0E37A13F036
:102F4000110F6AD1730764D43E0739D5384B9847BF
:102F5000C0F307230026A073E373030C000E237451
:102F6000E6726074DDF8148026776677A677E677D8
:102F700098F800002F4B214698470123A676E67665
:102F80002675667588F804300646C8B14046314655
:102F9000294BD8F82A90984700283FD10598013E40
:102FA000C0F80A604946254B984748B136E00028EA
:102FB00034D1E37AD8062ED4B10701D5DA072CD460
:102FC000059E3B07D6F82A3048BF47F02007EB6143
:102FD0002C62AF713078174B214698472861A37F48
:102FE000E27F1B0443EA0263227F00201343627FD7
:102FF000287243EA0223EB606872A872E8722876AE
:103000006876A876E8762E60F388AB8006E0092023
:1030100004E0082002E0042000E007200DB0BDE835
:10302000F08300BF41230000E92B0000952D000034
:10303000F11A000099220000552E0000E521000041
:103040002DE9F84F98460023C8F800304B4B044652
:103050000F4616469847002840F08E80A37919063F
:1030600000F18680DA0740F18680E568A368ED1AF2
:10307000AE4238BF3546002D77D0A368C3F30802AF
:10308000002A49D1206890F802B00BF1FF3B0BEA0F
:10309000532B1BF0FF0B0AD10BB9206902E06169C9
:1030A000374B9847012809D9431C42D06061D4F8B6
:1030B00000A061695046334B984720B9A37963F06B
:1030C0007F03A37154E06E0A00EB0B0922D09AF83B
:1030D000023006EB0B029A4288BFCBEB03069AF84C
:1030E000010039464A46F3B2DFF8A4C0E04700BB0E
:1030F00021680B7963B1D1F82A30C9EB0300B042E3
:1031000006D207EB40202E314FF400721E4B984739
:1031100076021FE0C4F81890A6682068C6F3080677
:10312000C6F50076A169194BB54238BF2E469847BF
:1031300030B1A379012063F07F03A371BDE8F88F5C
:10314000A1682368C1F30801194438462E3132467C
:103150000D4B9847A36837443344A360D8F8003038
:10316000AD1B3344C8F8003085E72846BDE8F88F2A
:103170000220BDE8F88F0720BDE8F88F6D2200001F
:103180007527000059270000D3210000E521000029
:103190007134000070B5214B05469847064600285B
:1031A00039D1AB799B0636D52868E9691C4B98471D
:1031B000064680BB2C6AE37A43F02003E372EB6897
:1031C0002377EB68C3F307236377EB681B0CA377C4
:1031D000EB681B0EE3772B69C3F30722A3761B0C66
:1031E00023751B0AE27663750E4B9847C0F30723DD
:1031F000A075E375030C000EA674E6742376607662
:10320000AB79012223F02003AB712B681A71286877
:10321000054B98470646304670BD00BF6D22000042
:10322000E5210000F11A00008526000010B5044BCE
:103230000446984718B920706070A070E07010BD07
:103240009531000070B594B014AB43F84C0D18469E
:1032500006A90122284B98470446002849D103AB10
:103260000C9306A80199254B98470446002840D1A5
:103270000B9E36B1F37A13F0010F0CBF0024072424
:1032800000E00624069B314618781D4B98470546FA
:10329000002C2ED1F37ADB0619D5012813D90DA8FD
:1032A00006A91C22174B98470DA80221164B0F9513
:1032B00098470446E8B90DA8144B9847044620B136
:1032C000042804D015E0022413E0072411E006A826
:1032D0000F4B9847044660B925B906980D4B98479F
:1032E000044606E0069829460B4B984704460028FA
:1032F000F3D0204614B070BD41230000E92B00003C
:1033000099220000D321000059280000FD2D000063
:10331000F128000085260000552E000070B59AB0F7
:103320001AAB43F8640D0E4618460CA901223B4B1C
:10333000984700286FD10C9B0CA81393019903ABFD
:10334000374C1293A047002865D11199002955D018
:1033500006A80B311522334DA84713A80CA91C222F
:10336000A84713A83146A047002849D0042852D1C5
:1033700013A82D4B984700284DD1189C132204F117
:103380000D000DF11A01A8479DF8183043F02003F5
:10339000E3720C9D01232B71159B0E9A9A4233D038
:1033A000E37ADB0630D52146204B28789847204B1E
:1033B000014628469847014620B31E4B28469847A9
:1033C0000C9B40BB93F84F202E2A1DD11A78032A5C
:1033D000159A04D1D3F822108A4208BF0022C2F302
:1033E000072183F86820120C83F86220120A83F800
:1033F0006320012283F869101A7105E004200AE0B5
:10340000082008E0022006E00CA80B4B984710B9F2
:103410000C980A4B98471AB070BD00BF41230000BA
:10342000E92B0000D3210000952D00009922000017
:1034300059270000E5210000F12800008526000042
:1034400008B528B9034B9847003018BF012008BDC4
:10345000012008BD9511000008B528B9034B984715
:10346000003018BF012008BD012008BD890C0000F4
:1034700070B50E4615461C4658B944B1294630462B
:10348000054B013C9847E4B205F50075F5E7204689
:1034900070BD042070BD00BF0110000070B50E4665
:1034A00015461C4658B944B129463046054B013CE7
:1034B0009847E4B205F50075F5E7204670BD042095
:1034C00070BD00BFBD10000010B51446C8B9042976
:1034D00004D8DFE801F0130A050C130001200EE008
:1034E000094B984780B2208004E0084B00E0064B6F
:1034F00098472060003018BF012000E00020C0B2D3
:1035000010BD042010BD00BFA90C00009D0C0000E0
:10351000024B13B10248FEF755B970470000000096
:103520002535000038B5094D094C641BA41018BF9F
:1035300005EB840505D0013C55F8043D9847002C67
:10354000F9D1BDE8384000F079B800BF4836000036
:103550004C3600000102006669726D776172652E5B
:10356000637572006669726D776172652E62696E4D
:103570000000000000C0092020C0092040C0092030
:1035800060C0092080C0092001000200040008007A
:10359000800000010002222A2B2C3A3B3C3D3E3F9A
:1035A0005B5D7C7F00809A90418E418F80454545D0
:1035B0004949498E8F9092924F994F555559999AF2
:1035C0009B9C9D9E9F41494F55A5A5A6A7A8A9AA2A
:1035D000ABAC21AEAFB0B1B2B3B4B5B6B7B8B9BA4F
:1035E000BBBCBDBEBFC0C1C2C3C4C5C6C7C8C9CAB3
:1035F000CBCCCDCECFD0D1D2D3D4D5D6D7D8D9DAA3
:10360000DBDCDDDEDFE0E1E2E3E4E5E6E7E8E9EA92
:10361000EBECEDEEEFF0F1F2F3F4F5F6F7F8F9FA82
:10362000FBFCFDFEFF000000F8B500BFF8BC08BCC5
:103630009E467047113500004D010000F8B500BFEF
:10364000F8BC08BC9E46704729010000000000003D
:10365000783600000000001090000000480B0000C9
:103660006CCAFF7F01000000F4E6FF7FB0B0B080BD
:0836700018E7FF7F01000000D4
:103678000000000064350000573500001201000208
:1036880000000040501D15604000010200010902C1
:103698001B0001010080FA0904000000FE0102037A
:1036A80009210BF40100020101040309041A035360
:1036B800006D006F006F00740068006900650057B6
:1036C80000610072006500120353006D006F006F07
:1036D8000074006800690065001A0353006D006FEC
:1036E800006F00740068006900650020004400460F
:1036F800005500000000F40100020000000E27073A
:04000003000000CD2C
:00000001FF
